:1000000012C02AC029C028C027C026C025C024C0CD
:1000100023C022C021C020C01FC01EC01DC01CC0E4
:100020001BC01AC019C011241FBECFEDCDBF10E0F8
:10003000A0E6B0E0E2E2F6E003C0C89531960D928A
:10004000A036B107D1F710E0A0E6B0E001C01D92E4
:10005000A036B107E1F731C0D3CFCF93DF93B92FEB
:10006000A82FF72FE62FD52FC42F8D919C91119794
:10007000CC9740F011961C921E928081918101963E
:100080009183808380819181CC9750F011961C924E
:100090001E921182108288819981019699838883AA
:1000A00088819981489730F01D921C9211821082AC
:1000B00019821882DF91CF910895C7EDD0E0DEBF9D
:1000C000CDBFAA24BB24B886AF82BE82AD82BC82DB
:1000D000AB82BA82A982DB2CCA2C4A2C5B2C6A2CFC
:1000E0007B2C8A2C9B2C2A2C3B2C8FE387BB8FE903
:1000F00081BB80E482BB88B38F6388BB80B39927C0
:10010000282F392F2072307085FF22C0919AA114B8
:10011000B104D1F48F819885019698878F83CC970D
:1001200099F4B886AF828D819E8101969E838D83DE
:100130004C2F5D2F4F5F5F4F6C2F7D2F6D5F7F4F7B
:100140008C2F9D2F059689DF21E0A22EB12C03C0B4
:100150009198A22EB32E91E0C916D10409F440C0A3
:1001600081E0C816D10430F092E0C916D10409F438
:100170006EC092C0949A9981909588B3892388BB68
:1001800091E0C92ED12C869928C04C0C5D1C84E0CE
:100190004816510459F489819A818C0D9D1D9A83CA
:1001A00089834C2F5D2F4C0D5D1D45C098E249168B
:1001B000510469F089E24816510408F46DC0952D88
:1001C000842D6FE070E017D2892B09F065C089811A
:1001D0009A8101969A8389832AC0442455245CC05D
:1001E000939A9B81909588B3892388BB82E0C82E1F
:1001F000D12C869929C00894611C711C94E0691661
:10020000710481F088E26816710461F099E2691660
:10021000710408F441C0972D862D6FE070E0EBD19A
:10022000892BD1F58B819C8101969C838B834C2FEC
:100230005D2F4F5F5F4F6C2F7D2F6D5F7F4F8C2F3A
:100240009D2F05960ADF28C06624772425C0929A40
:100250009D81909588B3892388BBCC24DD2480B30D
:100260009927282F392F2074307086FD13C00894E9
:10027000211C311C84E02816310471F40894811C7F
:10028000911C81E080BB93E08916910429F4822EB1
:10029000932E02C02C2C3D2C03E010E00819190904
:1002A000802F912FAA2797FDA095BA2F682F792F1D
:1002B0008A2F9B2FD8D017FF05C020E030E040E800
:1002C00057E472D020E030E04AE753E443D1E62E11
:1002D000F72E082F192F20E030E040E85FE3CDD063
:1002E00088231CF481E090E017C020E03FEF4FE747
:1002F00057E4912F802F7F2D6E2DC2D018161CF43D
:1003000080E090E009C0912F802F7F2D6E2D8ED040
:10031000B92FA82F972F862F0197F1F782B3837EED
:1003200082BB88B38F6388BB882D992DAA2797FD40
:10033000A095BA2F682F792F8A2F9B2F94D097FEE4
:1003400005C020E030E040E857E42ED020E030E067
:100350004AE753E4FFD0E62EF72E082F192F20E0AE
:1003600030E040E85FE389D088231CF481E090E02E
:1003700017C020E03FEF4FE757E4912F802F7F2DEC
:100380006E2D7ED018161CF480E090E009C0912FED
:10039000802F7F2D6E2D4AD0B92FA82F972F862F13
:1003A0000197F1F7ABCE5058192EA6D001D08CC0D2
:1003B000BA176207730784079507B1F188F40EF442
:1003C00010940B2EBA2FA02D062E622F202D072E53
:1003D000732F302D082E842F402D092E952F502D50
:1003E000FF275523B9F0591B49F0573E98F0469521
:1003F00037952795A795F0405395C9F776F0BA0F32
:10040000621F731F841F30F4879577956795B795A2
:10041000F040939517FA0F2E0895BF1BBB27BA0B18
:10042000620B730B840BF6CFDEF692C097FB70D095
:100430009F3738F0FEE9F91B982F872F762F6B2F07
:1004400005C083C09695879577956795F150D0F74D
:100450003EF490958095709561957F4F8F4F9F4F9B
:100460000895E89403C097FB0EF4F3DFB62F672FCF
:10047000782F892F9EE9002427C00ED05EF004C09B
:100480000BD026F001C008D019F020F48FEF0895AA
:1004900080E0089581E0089597FB092E052600F875
:1004A00068942DD0E89407FC07C06217730784078F
:1004B000950721F008F400940794989408959A956C
:1004C000BB0F661F771F881F11249923A1F0882373
:1004D000B2F79F3F59F0BB0F48F421F4002011F40C
:1004E00060FF04C06F5F7F4F8F4F9F4F881F9795AE
:1004F000879597F9089529C0052E092607FA440F14
:10050000551F5F3F79F0AA27A51708F051E04795DE
:10051000880F991F9F3F31F0BB27B91708F091E072
:10052000879508959F919F91112462C097FB880F32
:10053000991F9F3F31F0BB27B91708F091E08795CD
:1005400008959F919F91112453C06627772788278C
:1005500099270895D1DF01D0B7CF992339F05523DA
:1005600029F09F575F57950F13F4CAF1F1CF9158B7
:100570009F3FE1F3A62F00241124BB2766275527B0
:10058000F8E0A69520F4020E131EB41F651F220F7B
:10059000331F441F551FFA95A1F7F8E0E72F77277F
:1005A000F8E0E69520F4130EB41F651F7A1F330F91
:1005B000441F551FAA1FFA95A1F7F82F8827F69513
:1005C00020F4B40F651F7A1F8E1F440F551FAA1FFA
:1005D000EE1FFF23A1F788231AF4939539F408C07E
:1005E000000C111CBB1F661F771F881F0128089570
:1005F0009FEF80EC0895AA1BBB1B51E107C0AA1F07
:10060000BB1FA617B70710F0A61BB70B881F991FB3
:100610005A95A9F780959095682F792F8A2F9B2F4F
:0206200008953B
:00000001FF
